:020000020000FC
:1000000064C900000000000023C037C24FC10000D7
:10001000000052C1000000000000000002030406BE
:10002000080C101820304060800002030406080C01
:10003000101820304080FF000406080C10182030F3
:10004000406080A0C00005050D050D0603030302F6
:100050004FB662FD20C070FF1CC165FDFCC057FE9D
:1000600001C00994C0919700C395C0939700C5E063
:10007000C519B8F3D0919700CD1B98F3C8E7089441
:1000800083FDC795C4BDC52DCC2321F4C0E083FDFD
:10009000C0E8C4BD09C171FF03C0939894989598B6
:1000A000C52D089483FDC795C4BDC09399006B7F8F
:1000B000C52DCF3F09F443C0C0919800C395C093AC
:1000C000980070FF37C082FD05C09398949895986A
:1000D0004FBE18957860C091A000CC2391F0C091DC
:1000E0009800CA95D091A000CD1B58F0777FC091A1
:1000F0009800D0919F00CD1B08F41CC0209298005E
:1001000019C0939894989598C5E0CA95F1F7C09155
:100110007500CA95C2FD09C0C1FD05C095FFC19813
:1001200095FD92980EC0C2980CC095FF929895FDCF
:10013000C19807C09398949895984FBE18952092AF
:1001400099004FBE1895A5C0552021F095FF939AB0
:1001500095FD959A94989DC0552009F0949A95FF25
:10016000959895FD939895C0552021F095FF959A07
:1001700095FD939A95FF939895FD95988AC095FF64
:10018000929A95FDC19A95FFC19A95FD929AC5E004
:10019000CA95F1F7552021F095FF939A95FD959A10
:1001A000949877C095FF929A95FDC19AC29AC5E03E
:1001B000CA95F1F7552021F095FF939A95FD959AF0
:1001C000949867C0C29A95FF929A95FDC19AC5E02E
:1001D000CA95F1F7552009F0949A95FF959895FDE9
:1001E000939857C0C29A95FFC19A95FD929AC5E01F
:1001F000CA95F1F7552009F0949A95FF959895FDC9
:10020000939847C095FFC19A95FD929AC29AC5E00E
:10021000CA95F1F7552021F095FF959A95FD939A8F
:1002200095FF939895FD959834C095FFC19A95FDDB
:10023000929A95FF929A95FDC19AC5E0CA95F1F7F9
:10024000552021F095FF959A95FD939A95FF9398E7
:1002500095FD95981EC082FF1CC0C0917500C2FD1F
:100260000BC0C1FD11C095FF929A95FDC19A95FFF3
:10027000C19A95FD929A0DC0C1FDF5CF95FF929A56
:1002800095FDC19AC29A05C0C29A95FFC19A95FD83
:10029000929AC52DC095089483FDC795C4BDC0939F
:1002A00099002092970064604FBE18954FB6C0E148
:1002B000C8BF6E7F4FBE18953FB68F7EA9B7A0729C
:1002C000A2118061A9B7AF7DA9BFA9B7AE7FA9BFB1
:1002D0007894A0916600AA2349F0A92FAF7159F133
:1002E000A0916600AA95A093660025C040E050E06A
:1002F000A6B396FDA095A0FD4FEFAEB596FFA06406
:1003000096FDAF7BAEBDAA27A062A8BF8D7FA6B326
:1003100096FDA095A0FD5FEF451741F7A8E161FDAF
:10032000A0936600A92FAF7119F0A8E1A093660011
:1003300040938D008160A0916700AA2331F0A091C5
:100340006700AA95A093670007C0A92FAF7121F09D
:100350008061AA27A062A8BF80FF48C0A0918D003D
:100360004A2F8E7FA92FAF71C1F0403F08F040EFB8
:10037000A42FA295AF704A0F5091B000533069F08E
:10038000A695A69550FD01C0A69552FD03C0A41BDD
:100390004A2F03C04A0F08F44FEFA09196004A1766
:1003A00008F44A2F4093610071FF08C0A0916100DA
:1003B00050919200A51710F050936100A091610038
:1003C00040916300A41B70F04091CF00A40B50F04B
:1003D000A0916300A40FA093630040F4AFEFA0933B
:1003E000630004C0A0916100A0936300409163008A
:1003F000A09192004A1708F04A2F542EA52DA03440
:1004000008F06860A0916000A395A093600059F087
:10041000F894A9B7A160A9BF84FF03C0A9B7A062DF
:10042000A9BF3FBE189541E050916600552331F0B9
:10043000A92FAF7119F45A9550936600A0918D00C1
:10044000A13018F0209290000DC0209291002092CF
:100450009A00A0919000AF5FA093900018F0AFEFCA
:10046000A0939000F894A9B7A160A9BF84FF03C02E
:10047000A9B7A062A9BF3FBE18953FB646B557B50C
:100480008F7EA9B7A072A2118061A9B7AF7DA9BF65
:10049000A9B7AE7FA9BF789481FD28C0AEB596FFFD
:1004A000AF7B96FDA064AEBD8260A6B396FDA0951D
:1004B000A0FF05C0409364005093650036C1AEB5FF
:1004C00096FFA06496FDAF7BAEBDAA27A062A8BF31
:1004D0008D7FA92FAF7109F419C140E0A6B396FD35
:1004E000A095A0FD13C140938D0006C1AEB596FF47
:1004F000A06496FDAF7BAEBD8D7F61FF6CC0AEB5D5
:1005000096FFAF7B96FDA064AEBDAA27A062A8BFF0
:1005100082604093880050938900A09086004A1919
:10052000B09087005B09BB24A2E0EA2EA22C483CD5
:10053000A0E05A0730F4A0E1BA2EE22CAAE0AA2EDD
:1005400027C04836A1E05A0730F4A8E0BA2EE22CC2
:10055000AFE0AA2E1DC0403DA2E05A0730F4A4E04F
:10056000BA2EE22CAEE1AA2E13C0403AA5E05A07FB
:1005700030F4A2E0BA2EE22CACE3AA2E09C048392E
:10058000A8E05A0728F4A1E0BA2EE22CA8E7AA2E88
:10059000C42EA0918A00CA1AD52EA0918B00DA0A27
:1005A000DD202AF4AFEFC094D094CA1ADA0A209260
:1005B0008C00CA14DE0418F4A1E0A0938C004093D0
:1005C0008A0050938B00409188005091890040939D
:1005D000860050938700A09164004A1BA09165009B
:1005E0005A0B94FD7CC093FD7AC092FD76C056955F
:1005F000479591FD72C05695479590FD6EC0D52EDA
:10060000C42ED694C79461FD0CC0AC2DAC51AD2D59
:10061000A24008F07BC0DD2021F4AC2DA85C08F4DA
:1006200075C0A0E0EA2E97FD08C0E090C200A0913E
:10063000B400A33011F4E090CA00AAEFEA0EF22C45
:10064000F21CCE18DF084FB74170A091B400A33060
:10065000A9F4442329F095FD11C0F894906204C0D8
:1006600095FF0CC0F8949F7D939894989598929AD2
:10067000C29AC19A71FD01C060687894442369F000
:10068000A091B400A33031F4AFEFC094D094CA1A53
:10069000DA0A03C040E050E022C0A091B400A330C9
:1006A00049F4CC0CDD1CA5E0CA1AD20818F4A0E06D
:1006B000CA2ED22CAFEFCA16D20418F04FEF50E07A
:1006C0000EC0F090A700CF9C412D000C441F50E0BD
:1006D00008F012C04FEF50E00FC05695479594FFB9
:1006E00007C0552309F04FEFA42FA6954A0F521DBE
:1006F0004F3F520508F04FEF40938D00816061FF3E
:1007000005C0AFE1A095A923AB299A2FA8E1A0933A
:100710006600A92FAF7119F4AAE0A093660061FDED
:1007200004C0A92FAF7109F08F7EA6E0A0936700E7
:10073000A92FAF7119F4AAE0A0936700F894A9B7A4
:10074000A160A9BF84FF03C0A9B7A062A9BF3FBE33
:10075000189511E00AC013E008C01AE006C01EE1B7
:1007600004C014E602C018EC00C005E1BB27BA952E
:10077000F1F70A95D9F71A95C1F708952AE338E7F2
:1007800009C020E33CE806C02AE234EB03C025E2BE
:1007900038EC00C0652CB1E05B2E12E095FD9F7D2A
:1007A00095FF9062BB27C29ABA95F1F7552009F0E0
:1007B000949ABA95F1F79498BA95F1F7C298BA95C8
:1007C000F1F7552021F095FF939A95FD959AB091F8
:1007D000A800BA95F1F795FF939895FD9598B7E81D
:1007E000BA95F1F71A95D1F6022FB22FBA95F1F713
:1007F0000A95D9F73A9571F6C29A562C0895221B9C
:1008000039E0001F3A9509F40895221F211B18F4BE
:10081000210F8894F6CF0894F4CF622C722CB0E0AC
:100820008894B395221F331FE0F737952795889456
:10083000912E802E020B130B10F4192D082D10F49D
:10084000889401C00894661C771CBA9571F7172D1F
:10085000062D0895322D11232AF43A95009510950E
:10086000031B130BF894029F712C002D129F912CE7
:10087000802C7894780C172D921C292DB4E06B2EC7
:100880002695179507956A94D9F7332321F000959B
:100890001095031B130B0895089566FF21C0109156
:1008A00074001695009173000795B0917700B01B06
:1008B0000B2FB0917800B10B1B2F28F40038BFEF3D
:1008C0001B0740F009C00F37120508F405C00FE7F9
:1008D00010E002C000E81FEF00937C0010937D0041
:1008E000089566FF39C000917C00B09179000B0F2C
:1008F00010917D00B0917A001B1F20E030917D00A7
:1009000033230AF42A95B0917B002B1F1AF4203F61
:1009100040F00AC02F3008F407C00FEF1FEF2FE0A0
:1009200003C000E010E020EF30916300B09192002E
:100930003B1718F4332331F009C0B0917D00BB237D
:100940005AF004C0B0917D00BB2332F400937900CB
:1009500010937A0020937B00089566FF2FC02091AA
:10096000CD0000917C00000F10917D00111F72DFFF
:1009700011232AF40038BFEF1B0740F009C00F37DE
:10098000120508F405C00FE710E002C000E81FEFF1
:10099000002352F0B0916200B01B0B2F18F0013011
:1009A00008F00AC001E008C000950F5FB091620036
:1009B0000B0F08F001C00FEF00937E00089566FF53
:1009C0002DC02091CE0000917A0010917B0042DF73
:1009D00011232AF40130BFEF1B0740F009C00F3F7D
:1009E000120508F405C00FEF10E002C001E01FEF90
:1009F000112352F0B0917E00B01B0B2F18F0013084
:100A000008F00AC000E008C000950F5FB0917E00BA
:100A10000B0F08F001C00FEF0093630008950FEF74
:100A2000677FB72FB670E9F46860B0917400B83092
:100A300008F0677FB0917400A1F00FEF109174007F
:100A4000DEDEF894B09170000B9F112D002D78948C
:100A5000112309F00FEFB09195000B1710F40091DE
:100A600095000093940008956FC005D374FFB7E01C
:100A700074FDB6E0B068B064B7B9B6B1B068B06440
:100A8000B6B967DE74FFB7E074FDB6E0B068B06475
:100A9000B7B9B6B1B068B064B6B9B6B1B6FDFDCFFE
:100AA00004B115B1B6B1BF77B6B938D32AEB2093EC
:100AB000A30030E03093A400732E7694622E6694E7
:100AC000620E731E262D372D0217130778F08090C3
:100AD000A300BAEBB80DB093A3008090A400B0E0DF
:100AE000B81DB093A400260D371DEECF8090A30053
:100AF0009090A4001091A40016950091A300079572
:100B000016950795B091A300B00FB093A100B091D6
:100B1000A400B11FB093A20023E0169507952A9573
:100B2000E1F72091AF002A9529F42092A3002092AA
:100B3000A4000AC02A9521F0800E911E2A95E1F7A3
:100B40008092A3009092A40008952091AF00B6B1C6
:100B5000B6FDFBCF04B115B1B6B1BF77B6B9B09150
:100B6000A500B395B093A500B83060F12092A50020
:100B7000B091CC00BB2321F1112329F0B091A60044
:100B8000BF3F61F009C0B091A6000B1739F020F407
:100B9000BB2321F0BA9502C0B395E1F30091920016
:100BA000B093A600B93B50F400ECBA3A38F400E830
:100BB000BB3920F400E4BC3808F400E00093920054
:100BC0007F7E0895B0919200B39511F0B09392009A
:100BD000B091A500B73009F47061089502E3F8946C
:100BE000B091D0000B9F012D000C001F7894B091A4
:100BF00092000B1710F00091920000936100009397
:100C00006300502E00939500089520927300B8E081
:100C1000B093740008952091800030918100F89481
:100C20000CB51DB5200F311F3BBD2ABD6160B0E181
:100C3000B8BF7894209171003091720000937100D8
:100C400010937200021B130B2091730030917400FB
:100C5000622E732EB4E08B2EB2E09B2EB091740006
:100C6000B43010F08A949A94B83010F08A949A9420
:100C7000769467948A94E1F726193709992021F030
:100C8000169507959A94E1F7200F311F2093730072
:100C90003093740008F00895BFEFB0937300B093E1
:100CA000740008952091820030918300F8940CB56F
:100CB0001DB5020F131F1BBD0ABD6160B0E1B8BFB7
:100CC0007894089560FDFECFEDDF0895B091BE00E9
:100CD00000916E00023808F0B395003A08F0B39521
:100CE000B63008F0B5E09B2EBCE08B2EB0917400BE
:100CF000B33030F48394839482FF02C0839483944E
:100D0000B23030F48394839482FF02C0839483943E
:100D100071FF03C0B3E09B2E822C109174000091F0
:100D2000730024E0169507952A95E1F70819120932
:100D300028F0B02FB250B12FB20910F402E010E049
:100D4000312F202F712E602E76946794B92DB330F9
:100D5000E9F0B0FD05C0060D171D262D372D06C084
:100D6000000F111F0250120922E030E0B92DB330FC
:100D700068F02093840030938500009380001093E6
:100D80008100609282007092830008950093840035
:100D90001093850020938000309381006092820040
:100DA00070928300089560FDFECF20918200220F93
:100DB00030918300331FB72FB67021F0209173005C
:100DC00030917400F8940CB51DB5020F131F1BBDB4
:100DD0000ABD6160B0E1B8BF789408956061209267
:100DE000760020E004C060612092760020E2B72FF8
:100DF000B67009F06F7E789460FD05C0B091760002
:100E0000BB2309F0089501E063FF0AC0B0917400AC
:100E1000B33008F002E0B0917400B63008F003E09F
:100E200071FF01C006E060FD06C0B0917600BB23F3
:100E300011F0789408951AE083FF1AE07894000086
:100E40000000F89462FD03C014E183FF14E171FF18
:100E500001C018E7B4B530919900B31BB10B18F37A
:100E6000B0917600B395B0937600B5E03B2F6B2E32
:100E7000722CB8B1B072B21709F073943A95C9F7F1
:100E80007394761488F464FFB2CF6F7E3CB56DB472
:100E90007090730080907400370D681C6BBC3ABD75
:100EA0006160B0E1B8BFA3CF64FDA1CF0A9509F09E
:100EB000BACF7894089571FF0AC0B0916D00B395D0
:100EC000B0936D0060FD0CC020926D0009C060FD04
:100ED00007C064FD05C067FD03C0BF91BF91BAC4E0
:100EE00008952091840030918500F8940CB51DB5CB
:100EF000020F131F1BBD0ABD6160B0E1B8BF78943B
:100F00000895EFDF00E063FF03C064FF01C001E06C
:100F1000F89410916E00B7E01B9F212D102D78944E
:100F2000200F2695179526951795269517951093BA
:100F30006E00183718F4B8E7B0936E0000916E0099
:100F4000B0916F000B1720F0606293989498959879
:100F500060FDFECF0895F894929AC29AC19A82FFDA
:100F600007C0E2E0F1E073FF03C0B5E0BA95F1F726
:100F7000B0917400BC7F81F0552021F095FF939AC9
:100F800095FD959AB6E0BA95F1F795FF939895FD82
:100F90009598B5E0BA95F1F795FF929895FDC198AF
:100FA000B2E0B0937500ABC0F89495FF959895FDAD
:100FB000939882FF0DC0E2EFF0E073FF0BC0C29A7E
:100FC00095FFC19A95FD929AB5E0BA95F1F702C0E6
:100FD000ECEAF0E062FF03C0552009F0949AB3E018
:100FE000B09375008CC0F894929AC29AC19A82FF0D
:100FF00007C0E2EEF0E073FF03C0B5E0BA95F1F789
:10100000B0917400BC7F81F0552021F095FF959A36
:1010100095FD939AB6E0BA95F1F795FF959895FDF1
:101020009398B5E0BA95F1F795FFC19895FD929820
:10103000B4E0B093750063C0F894949882FF0DC03B
:10104000E2EDF0E073FF0BC095FF929A95FDC19A17
:10105000C29AB5E0BA95F1F702C0E4EAF0E062FFA7
:1010600006C0552021F095FF939A95FD959AB5E01D
:10107000B093750044C0F894929AC29AC19A82FFC4
:1010800007C0EFEBF0E073FF03C0B5E0BA95F1F7EE
:10109000B0917400BC7F51F0552009F0949AB6E0ED
:1010A000BA95F1F79498B5E0BA95F1F7C298B6E021
:1010B000B093750024C0F89495FF939895FD95988A
:1010C00082FF10C0E5E1F1E073FF0EC095FF929A38
:1010D00095FDC19A95FFC19A95FD929AB5E0BA9592
:1010E000F1F702C0E4EBF0E062FF06C0552021F00A
:1010F00095FF959A95FD939AB1E0B093750067FFBF
:101100000AC00CD0B5E0BA95F1F7B5E0BA95F1F7A1
:101110009298C298C1986F7D7894089523EA30E040
:10112000F901939894989598929AC29AC19A6B7F74
:101130000895ACEAB0E00FEF0D930D930D930D936E
:1011400003E00D9304E00D930BE00D9303E00D938A
:1011500001E00D9301E00D93A8EBB0E001E00D93E9
:101160000FEF0D930D930FEF0D930D930D9303E080
:101170000D9306E00D930FEF0D930D9305E20D9384
:1011800000ED0D930AEF0D930AEF0D9304E00D931C
:101190000DE00D9301E00D9300E00D930AE70D9330
:1011A0000FEF0D9301E00D9308952091BF0009E02A
:1011B00011E0223011F405E011E0233011F405E0D4
:1011C00012E0243011F405E013E0253011F409E0B9
:1011D00017E0263011F400E010E000939F00109318
:1011E000A0002091B3008B7F233009F48460777FC7
:1011F000233009F47860B091B400B33019F09F7DCA
:10120000B1FD90629F7BB091B500B1FD9064B22FAB
:10121000B23011F0886001C0877F0895ECE1F0E002
:101220000091AC000A95E00FF21DB491B093CD008F
:101230000091AD000A95E00FF21DB491B093CE007D
:101240006DDF0895EAE2F0E00091C7000A95E00F33
:10125000F21DB491B093CF0061DF0895E8E3F0E0B0
:101260000091B2000A95E00FF21DB491B093D00046
:1012700055DF08950895B091C8000FEF1CE0B2301B
:1012800011F400EA1AE0B33011F402E815E000931B
:101290006F0010937000089508952091C20030915E
:1012A000C30097FF02C020E03FEFB32FB21B6B2EAD
:1012B000B25810F4B2E86B2E00E00395609EB12D99
:1012C000B058D8F30093A7000895F894E3E0F0E055
:1012D000B9E0B7BFB491B078C1F3F894A895B1B5AF
:1012E000B861B1BDB0E0B1BDB4E0BEBFBFE5BDBF48
:1012F00015DFB6E0B8BBB6E1B7BBB0E0B5BBB0E058
:10130000B4BBB4E0B2BBBCE3B1BB2224A0E0B0E00C
:101310002D92AA31E9F7A0E6B0E00FEF2D920A95E1
:10132000E9F707DFB7D241DF79DF8CDF97DFA2DF94
:10133000A2DFB2DFB2DF0091C4000093A800EEDEAE
:10134000B2E0B3BFB2E0BEBDB2E0B5BDF8940BDA17
:1013500015DA05DA16DA03DA17DA01DA26D303DA50
:1013600002DAFFD9B1E5B8BFB9BFB0B7B860B0BF56
:10137000B6B1B460B6B9EDD9789476DBB9B7B062DE
:10138000B9BFBB27B062B8BF8D7FEDD9B1E0B093D4
:101390006900626025E0B0918C00BB2309F425E070
:1013A000DAD9B0918D00B230A8F3B92FBF71009196
:1013B0008F0000938E00B0938F00B01759F72A95D5
:1013C00051F76D7FBEB596FFB06496FDBF7BBEBD85
:1013D000BB27B062B8BF8D7FC4D9BDD902E0B92F99
:1013E000BF7109F400E0B0918D00B017B0F3F8942C
:1013F000C5D9C4D9C3D97894B6D920927F00B09109
:10140000B400B33009F472C0A6D9B091B800B130BD
:1014100008F46CC0B0916900B13008F467C0B92F0E
:10142000BF71C1F0B0918D00BF3F08F45FC0F89468
:10143000AED9789496D9B0918D00B130C0F7F894B8
:101440009DD98BD99BD978948CD9B0918D00BF3F11
:10145000B0F3DDC2B8E09B2E9068F8941EDF78945C
:1014600080D9F8949F7719DF80908D00B0918D001E
:10147000BF37789408F442C06CD9F89488D978942E
:101480009A9451F7B82DB550B093C3006CD9F89425
:101490002ED290D27894BAE09B2E9068F894FDDE1C
:1014A00078945FD9F8949F77F8DE80908D00B091A2
:1014B0008D00BF37789478F74CD9F8945FD94DD91F
:1014C0005DD978949A9449F7B82DBB5FB093C20068
:1014D0004AD9F8940CD27DD2789443D9F894DDDEC1
:1014E0007894B0918D00BF3FC0F391C200918D0000
:1014F000B0917F000B1710F000937F0032D901E00C
:10150000B091B400B35009F405E0B0918D00B0176C
:1015100008F075CFF8943BD93AD939D9789423D9C2
:101520002092690020926A0020926B00B0916A00BC
:10153000B395B0936A00BF3F69F5B0916B00B39566
:10154000B0936B00B091C60009E1BA9559F002E37F
:10155000BA9541F00DE7BA9529F00AEFBA9511F066
:1015600020926B00B0916B00B017A0F0B0916B00AF
:10157000BA95B0936B00B4EBB0936A00B091C5001C
:10158000B093A800F89403D97894B091C400B093B4
:10159000A800E7D8E2D8B0916600BB2321F4B92FA8
:1015A000BF7109F4F6CEB0918D00B63008F4BECF0D
:1015B000B091B400B35009F0D4D8B0916600BB2309
:1015C00009F4E7CEF894AADD20926100209262002F
:1015D00020926300522C7894B091B100B0939600A1
:1015E00020927700209278002092790020927A0051
:1015F00020927B002092A50060E070E020926E00B7
:1016000004DBB8E0B093A5007061A3D874FFB7E025
:1016100074FDB6E0B068B064B7B9B6B1B068B06494
:10162000B6B9B6B1B6FDFDCF04B115B1B6B1BF774D
:10163000B6B9112309F00FEF0093A60086DAB8E0DF
:10164000B093A50070618090B300B2E0B093B30096
:10165000ACDD8092B300F894BFEFB0939200BEDA95
:10166000B0916100B0939200B0939300B093940056
:101670007894B1E0B0936100B09363005B2EB093B7
:101680009B00B0919100B0939A00716072602092BB
:101690006D00F1DC10DDBFDAB8DA18DB04C085DDDF
:1016A0002092A5007F7E95FF04C0B0B7B77FB0BF82
:1016B00007C0B0B7B860B0BFB0E0B068B064B7B949
:1016C00092DBF9DB0EDCE8D81CDC45DCA4DAFADAC4
:1016D000FDDA69DBB0B7B860B0BFB1E0B068B06444
:1016E000B7B97CDBE8DBFDDBD8D899D90ADC5CDC58
:1016F00092DAE8DAEBDA57DB95FF08C0B0B7B860EA
:10170000B0BFB0E0B068B064B7B903C0B0B7B77FDE
:10171000B0BF69DBD0DBE5DBE4D8F3DB64DC7BDA8C
:10172000D1DAD4DA40DB95FF04C0B0B7B77FB0BFE1
:1017300007C0B0B7B860B0BFB0E0B068B064B7B9C8
:101740004DDBB9DBCEDB09D9DCDB76DC64DABADA77
:10175000BDDA29DBB0B7B860B0BFB1E0B068B06443
:10176000B7B941DBA8DBBDDB2AD9CBDB84DC53DA9C
:10177000A9DAACDA18DB95FF08C0B0B7B860B0BF23
:10178000B0E0B068B064B7B903C0B0B7B77FB0BF5E
:1017900025DB74FFB7E074FDB6E0B068B064B7B99C
:1017A000B6B1B068B064B6B986DB9BDBAADB83DC7C
:1017B00032DA88DA8BDAC9D9F6DA71FF25C067FD2B
:1017C00023C0B0919500B0939200B0939300B09174
:1017D0009100B0939A00B1E0B0939B0014E624E12D
:1017E000B0916D00B11750F07D7F746020936C0054
:1017F000BFEFB0939200B093930006C0B0918D00FC
:10180000B13008F050CF26C072FF10C067FD0EC087
:10181000B0916C00BA9511F47B7F41CFB0936C000E
:10182000B0918D00B13008F03ECF14C0B09190005F
:10183000B23880F4B92FBF7121F4B0916600BB2398
:1018400049F0B091740000EF67FF01C000E6B017E7
:1018500008F429CFF89462DC8090B300B2E0B09332
:10186000B300A3DC8092B30020926100209262005A
:1018700020926300522C209296007E7F789469D744
:101880004DDCB92FBF7129F4B0916600BB2309F478
:1018900080CD48CEEDE0F0E023D00A3509F01BC042
:1018A000EEE0F0E01DD0053A09F015C03AE0ACEAF0
:1018B000B0E0E3E0F0E014D00D9331963A95D9F71B
:1018C00035E1A8EBB0E0EFE0F0E00AD00D933196FF
:1018D0003A95D9F702C02DDC0AD0E4E2F0E0089591
:1018E000E199FECFEEBBFFBBE09A0DB308951ED089
:1018F0003AE0ACEAB0E0E3E0F0E00D910FD03196D1
:101900003A95D9F735E1A8EBB0E0EFE0F0E00D91C2
:1019100005D031963A95D9F712D00895E199FECFC6
:101920000DBBEEBBFFBBE29AE19A0895EDE0F0E05B
:101930000FEFF4DFEEE0F0E00FEFF0DF0895EDE001
:10194000F0E00AE5EBDFEEE0F0E005EAE7DF08951E
:101950003091A9000091AA00313011F40093B00039
:10196000323011F40093B100333011F40093B2001F
:10197000343011F40093BE00353011F40093C700E9
:10198000363011F40093BF00373011F40093B300E8
:10199000383011F40093C800393011F40093B400CA
:1019A0003A3011F40093B500089525E0DCD62A956D
:1019B000E9F70895E3D6E5D6E7D6E9D6CED6DED662
:1019C000E0D6E2D6E4D6C9D6D9D6DBD6DDD6DFD688
:1019D0000895DDD6D9D6D5D6D1D6BFD6D8D6D4D6C9
:1019E000D0D6CCD6BAD6D3D6CFD6CBD6C7D60895F6
:1019F0008090A9009090AA00C1D6C0D6BFD6ADD61F
:101A00008A94D1F7C4D6A9D69A94E1F70895F894A8
:101A1000D1DF7894CADFC9DFB1E0B093A900B1E0AB
:101A2000B093AA002092AB00F894E2DF7894B5E07E
:101A30006B2E70908D0097D6B0918D007B16C9F7F4
:101A4000B13018F0BF3F40F107C082DFF8944FDF9C
:101A5000B1DFB8E0B1BDA9DF6A9459F7B091AB002E
:101A6000B395B093AB00B33008F4DECF9EDFB091F6
:101A7000AA00B395B093AA00F894B091A900BA95C2
:101A8000E6E4F0E0EB0FF21D049178940395B09139
:101A9000AA00B01708F4C6CF88DF87DFB091A9008D
:101AA000B395B093A900B091A900BB3008F4B7CFAB
:0C1AB00040DBF8941CDFB8E0B1BD77DF2C
:00000001FF
